:020000021000EC
:10F800000C9446FC0C9463FC0C9463FC0C9463FC19
:10F810000C9463FC0C9463FC0C9463FC0C9463FCEC
:10F820000C9463FC0C9463FC0C9463FC0C9463FCDC
:10F830000C9463FC0C9463FC0C9463FC0C9463FCCC
:10F840000C9463FC0C9463FC0C9463FC0C9463FCBC
:10F850000C9463FC0C9463FC0C9463FC0C9463FCAC
:10F860000C9463FC0C9463FC0C9463FC0C9463FC9C
:10F870000C9463FC0C9463FC0C9463FC0C9463FC8C
:10F880000C9463FC0C9463FC0C9463FC11241FBE69
:10F89000CFEFD0E1DEBFCDBF11E0A0E0B1E0E8E402
:10F8A000FFEF01E00BBF02C007900D92A030B1073F
:10F8B000D9F712E0A0E0B1E001C01D92A434B10775
:10F8C000E1F70C9466FF0C9400FC0F92AF93BF938A
:10F8D000CF93DF93EF93FF93FC01EA01DB01D8950F
:10F8E000099231961197D9F7FF91EF91DF91CF915E
:10F8F000BF91AF910F9008950F921F920F93AF9306
:10F90000BF93CF93DF93EF93FF93FC01EA01DB01F9
:10F910000990199001E043D032961297C9F7FC0183
:10F9200003E03DD005E03BD0FF91EF91DF91CF9117
:10F93000BF91AF910F911F900F9008950F931F9358
:10F94000EF93FF93FC0103E02AD000E011E0E00F09
:10F95000F11FE617F707B9F7FF91EF911F910F918C
:10F9600008950F930F9222D0082E09E018D00F901F
:10F970000F9108950F930F92EF93FF9317D0FC010F
:10F9800060936800C895802DFF91EF910F900F91C3
:10F9900008950F930BD001E102D00F910895E199E2
:10F9A000FECF00936800E895FFFF0000009168001B
:10F9B00000FDFCCF089587E089B98AB188618AB9D2
:10F9C00008958AB1877E8AB908958CB95E9BFECF6F
:10F9D0005E9A08958CB1992708958BB19927807804
:10F9E00090700895EF92FF920F931F93CF93DF9340
:10F9F0007B01C0E0D0E0C617D70770F48C010E94ED
:10FA0000EDFC8823E1F30E94EAFCF80181938F0169
:10FA10002196CE15DF0598F381E090E0DF91CF913C
:10FA20001F910F91FF90EF900895EF92FF920F9327
:10FA30001F93CF93DF937C018B01C0E0D0E0C01710
:10FA4000D10738F4F70181917F010E94E5FC2196EE
:10FA5000F6CF81E090E0DF91CF911F910F91FF9061
:10FA6000EF90089540E050E04817590750F422E520
:10FA700037E000002150304037FFFBCF4F5F5F4F32
:10FA8000F3CF08950E94E1FC0E94000008950E94B7
:10FA9000EDFC8823E1F30E94EAFC803219F481E056
:10FAA00090E0089585E10E94E5FC80E090E00895F3
:10FAB00090E0282F33272138310589F0223831058D
:10FAC00024F42038310549F00DC02238310549F0C1
:10FAD0002839310539F493E005C092E003C091E084
:10FAE00001C092E1892F9927089540E050E060918C
:10FAF00040017091410146175707D0F4209142020E
:10FB000030914302E2E4F1E03FBB2EBB2F5F3F4F59
:10FB100080818DBBE29AE19AE199FECF4F5F5F4F02
:10FB200031964617570780F33093430220934202E1
:10FB3000089540E050E06091400170914101461706
:10FB40005707B0F42091420230914302E2E4F1E021
:10FB50003FBB2EBB2F5F3F4FE09A8DB381934F5F2A
:10FB60005F4F46175707A0F330934302209342029A
:10FB70000895CF93DF93809142029091430297FFC3
:10FB800003C081E08BBF01C01BBEC0E0D0E080910C
:10FB9000400190914101C817D907A0F4CE018E5BB6
:10FBA0009E4F2091420230914302220F331FAC013D
:10FBB00060E071E0C9018C0F9D1F0E947CFCC05069
:10FBC000DF4FE5CF0E94C9FCDF91CF9108952091CE
:10FBD00042023091430237FF03C081E08BBF01C076
:10FBE0001BBE42E451E06091400170914101C901A6
:10FBF000880F991F0E9465FC0895CF93C0E069E0CB
:10FC000081E090E00E94BAFC992784FF03C08F7EB8
:10FC10000E94B1FC0E94EDFC8823E1F30E94EAFC03
:10FC20009927823591051CF5803591050CF05CC053
:10FC30008134910509F462C0823491057CF48133EA
:10FC40009105B1F18233910524F4C09709F44CC0B9
:10FC500037C18034910509F437C132C1823491052E
:10FC600009F45FC08534910509F45EC029C1863569
:10FC7000910509F4F0C0873591054CF48235910562
:10FC800009F45FC08535910509F468C019C184374E
:10FC9000910509F4A3C0853791052CF484369105AC
:10FCA00009F475C00DC18537910509F4C4C008C1B8
:10FCB0000E9447FD882309F4ADCF84E10E94E5FC52
:10FCC00081E40E94E5FC86E50E94E5FC82E50E9455
:10FCD000E5FC80E20E94E5FC83E50E94E5FC84E50A
:10FCE0000E94E5FC8BE406C00E9447FD882309F4CE
:10FCF00091CF84E10E94E5FC80E1E3C061E070E027
:10FD000080E091E00E94F2FC0E9447FD882309F404
:10FD100081CF84E10E94E5FC809100010E9458FDA2
:10FD2000E9CF64E170E008C061E070E080E091E05C
:10FD30000E94F2FC64E070E080E091E00E94F2FC3E
:10FD4000D3CF0E9447FD882309F464CF60E070E0C0
:10FD5000CB010E949EFC0E94C9FCCBCF62E070E008
:10FD600080E091E00E94F2FC0E9447FD882309F4A4
:10FD700051CF20910001809101019927982F882768
:10FD8000820F911D9093430280934202B2CF63E0B1
:10FD900070E080E091E00E94F2FC209101018091EE
:10FDA00000019927982F8827820F911D9093410178
:10FDB00080934001BC0182E491E00E94F2FC0E9429
:10FDC00047FD882309F426CF80910201863419F477
:10FDD0000E94B9FD8ECF0E9475FD8BCF63E070E06D
:10FDE00080E091E00E94F2FC2091010180910001ED
:10FDF0009927982F8827820F911D90934101809316
:10FE000040010E9447FD882309F404CF809102013C
:10FE1000863419F40E94E7FD02C00E9499FD84E136
:10FE20000E94E5FC609140017091410182E491E003
:10FE30000E9415FD61CF0E9447FD882309F4EACE98
:10FE400084E10E94E5FC8EE10E94E5FC87E90E94C6
:10FE5000E5FC82E04FCF64E070E080E091E00E943A
:10FE6000F2FC0E9447FD882309F4D4CE84E10E946D
:10FE7000E5FC80910001803531F4809101018823F7
:10FE800061F4C82F17C0883531F4809101018830A2
:10FE900061F4C3E00FC0803531F4809101018830F6
:10FEA00049F4C2E007C0883529F480910101882314
:10FEB00009F4C1E069E08C2F99270E94BAFC1ACF9F
:10FEC00085E10E94E5FCA6CECF910895CFEFD0E169
:10FED000DEBFCDBFCEE1F894AEEFBFE00E949BFF46
:10FEE000802D843B79F4AFEFBFE00E949BFF802D13
:10FEF000833C41F4ADEFBFE00E949BFF802D99272A
:10FF000080936F000E94DBFC0E94EAFC84E690E094
:10FF10000E9432FD0E94EDFC882319F00E94FDFD35
:10FF200004C0C150C8BBCC2389F70E9442FD80E0C9
:10FF300090E00C94A3FFE199FECFBFBBAEBBE09A6B
:08FF400011960DB20895FFCFE8
:040000031000F800F1
:00000001FF
